:100000008B018316FC30E9298C00030E83018D00DF
:1000100004088E000F0884008001061F80170F0857
:100020004E3A173003198F0003100016061F0314F1
:10003000800C1A280000031C1628061B0310800CD5
:100040008C0E800C8F0A24280000061F80170008E1
:1000500096070E0884000D0E86080B1083000C0E08
:100060000900120881010B11900003103908820762
:10007000B628BA28BE28C328CE28E128150882074A
:100080004A2A0D2967281808DF39FC3E03185F2823
:10009000043E82075C285C285C28612818080F3918
:1000A000F93E03185F28073E8207562B622B742BFC
:1000B000902B9D2BA52BAA2B95002130B5298230A2
:1000C000B5290130B5210430B521FB30B5291A30EE
:1000D00084002D3090008001840A900B6B283A1523
:1000E00022308400043092003918862800008619D6
:1000F0009528861995288619952886199528861990
:10010000952886199528861995289928861D952859
:10011000861D9528861D9528861D9528861D95285F
:10012000861D9528861D952899283120013092003A
:1001300074281208CA21013E9200031C74283B3027
:100140008400CD21A000CD21A100CD219E00CD2194
:100150009F00B801183090001A3084000008B802DF
:10016000B521840A900BAE283808B52910089C00E8
:10017000B90AC82810089D00B90AC8281008A000AC
:100180009B0AB90AC92810089E009B0AB90A0000F8
:1001900000000000B221C921B4210800B90A1008EA
:1001A0002002F420031DDB282008BB070318BC0A2B
:1001B000BD0A00000800A100BE070318BF0AC00A5C
:1001C0000800B90310081E02F420031DEE281E08C3
:1001D000C1070318C20AC30A000008009F00C40731
:1001E0000318C50AC60A0800031C003CF83E031C9D
:1001F0009001030103183A0880040310BA0D031C90
:100200000B29840A0408323A2230031984003A1474
:100210009B0A10080800A02108291108A421100831
:10022000A2210430920006301729083017299700C0
:1002300086192229970B18291208013E92000318EB
:10024000352915291208A2210230920006302A29E8
:1002500008302A299700861D3B29970B2B29120865
:10026000013E9200031835292829013091000230FF
:100270009000FF30A42912081029FE308C00981E2F
:1002800044291C309B078C001C089200970117140E
:100290000B1140308F0021308400303006048D0077
:1002A00000008C0A0D08860403108F0D03188F0AB6
:1002B0000318840A90010F080005031D900ACF302F
:1002C000860504088E001E300C1C203010078400A8
:1002D000181B6A29981B6C290D088604981E76291C
:1002E00000000C088400000890007C2900088C1B8A
:1002F0001D0890000E088400981B7E29CF308605CB
:10030000013097060319920303198F29181B8829B6
:10031000981B8A290D0886049F2100007C2910085B
:10032000920017140B1130308D061B080C06031DAC
:100330005129CF3086051C30981A9B020800A0294D
:100340000800010881010B1197000B309200031087
:10035000031CAC298613AE2986170314970C920B45
:10036000A8290800B42900009F291418A429900086
:100370000B3092000310060880380318803A86007C
:100380001F309100910BC2290314900C920BBB29D2
:100390000800B229C921B321080000089900840A85
:1003A00000089A00840A00089B00840A9001900AC1
:1003B00003101B0C990703189A0A0310990D9A0D44
:1003C0001B081A0203189A00900D031CDE2910085E
:1003D0000800850049308600C530810083128601FF
:1003E00006090139CF008501880194019501F8299A
:1003F000412381010B11150BFE29062A18300F0627
:10040000031DC12A861DF9290B1DFE298101183003
:100410000F06031DC12A060801394F06031D1C2AB9
:10042000861D192A011E072A153090070318910A04
:10043000062A8B133E20F8298B139000930192011A
:100440000314920D10081205031D282A930A212A6D
:10045000CF064F050830031D803E1307A500FF306F
:10046000A000A100A200A300A400890188012530FA
:1004700084009922F82914104F30B5214B30B52152
:1004800081010B11861D402A0B1D422A8619462A1E
:100490004A22402A81010B111D308400093091004D
:1004A0008001840A910B502A9D0A2030840086190D
:1004B0005C2A0B1D572A642A01081E029E02A522EF
:1004C000861DA02A0B1D602A2508F03E031C08008B
:1004D0001D08800625308400E8302006CA30031944
:1004E000A000D5302006C1300319A0008901831671
:1004F0000814831200080806031D8F2A890A840342
:10050000841A772A83160814831208089100890A2E
:10051000831608148312C62325308400992A2530B7
:1005200084000908083EF8398900891E772A890164
:1005300088010008B5218403841A992AB923080088
:1005400001081F029F02A522572A81010B1190006A
:10055000901B003CFB3EA50A9D0D031C08001D08D6
:10056000800601309D00840A25300406031D080022
:100570002208A1002308A2002408A3008403A401E8
:1005800008001430910081010B1118081F39333015
:1005900003194930981ECF2A1A30181A19070F0666
:1005A0000319DA2A0B1DC52A910BC42A8B1381303B
:1005B000B521F8298B1380309608031DD82A981A84
:1005C0003B2BE322F8292030B521491018081F39A8
:1005D00093000319930A3D2119080F3997001A084F
:1005E0009200120817040319FE2ACA21C92100002B
:1005F000F92A9203120903199703F12A930BEB2AA4
:1006000018081F390319062B491C372BB21E112B52
:10061000B212320898001F390319980AE030B20567
:1006200049141630930018309200323097001708A2
:10063000840000088E0012088400000890000E0854
:1006400080001708840010088000920A970A930B14
:10065000172B18081F39491C342B0319E62A980355
:10066000FF3E031DE62A372B0319980AE62A0608DF
:10067000CF3986000800181E3F2B4E20F829432052
:10068000F8291414960118308F00990186088B01FF
:100690008B158B1708005023502350235023502BC9
:1006A000B23081000B110B1D532B08000430B52113
:1006B0000330B5210630B5210030B5210030B52119
:1006C000F330B5291A0D8900890D890D0830930082
:1006D000B801831608148312890A0808B802B521E4
:1006E000930B692B3808B5291A0D8900890D890DDE
:1006F000083093001B30840000088800831608121D
:10070000081555308900AA3089008814081E862BE8
:1007100008118312890A840A930B7C2B2130B52996
:10072000B8010508B802B5210608B802B5210030A5
:10073000B5210030B5213808B5292030B5211A0877
:1007400091001B088800C623B92B06090139CF0088
:100750002130B5290430190292001C3E84000008A3
:10076000980098161A0899001B089A0012089B0016
:10077000E32A88080319BF2B5023880BBC2B0530B4
:1007800084009119840A09098005080007301105C1
:100790009200920A97010314970D920BCC2B05300F
:1007A00084009119840A1708911FDD2B111B800604
:1007B0001709111F80058901E12B8004111B0030EE
:0407C00089000800A4
:10400000FF3FFF3FFF3FFF3FFF3FFF3F6005FA3F9E
:1042000000000000000000000000000000000000AE
:10421000000000000000000000000000000000009E
:10422000000000000000000000000000000000008E
:10423000000000000000000000000000000000007E
:10424000000000000000000000000000000000006E
:10425000000000000000000000000000000000005E
:10426000000000000000000000000000000000004E
:10427000000000000000000000000000000000003E
:00000001FF
